:020000040000FA
:1000000028EF08F01200000007EF00F01200DACF2E
:10001000E4FFE2CFDAFFE6529EA218D09E920001E2
:10002000A22BA2A112D0010EA36FD59E8D1DD76E5B
:100030008C1DD66EF294D58E818C818ECD90FE0E65
:10004000CF6E6F0ECE6E9E90CD80A4D0F2A49FD0C6
:10005000F294D59E0001A351080A01E18DD00F0A48
:1000600001E179D0010A65E0030A51E0010A3DE0AF
:10007000070A29E0010A15E0030A01E086D0819C05
:10008000D59E8F1DD76E8E1DD66EF294D58E818A29
:10009000818ECD90FE0ECF6E6F0ECE6E9E90CD8077
:1000A00074D0819AD59E911DD76E901DD66EF29414
:1000B000D58E8188818ECD90FE0ECF6E6F0ECE6E66
:1000C0009E90CD8062D08198D59E931DD76E921D53
:1000D000D66EF294D58E8284818ECD90FE0ECF6E38
:1000E0006F0ECE6E9E90CD8050D08294D59E951D81
:1000F000D76E941DD66EF294D58E8282818ECD906D
:10010000FE0ECF6E6F0ECE6E9E90CD803ED0829250
:10011000D59E971DD76E961DD66EF294D58E828889
:10012000818ECD90FE0ECF6E6F0ECE6E9E90CD80E6
:100130002CD08298D59E991DD76E981DD66EF294BC
:10014000D58E8286818ECD90FE0ECF6E6F0ECE6ED6
:100150009E90CD801AD08296D59E9B1DD76E9A1DFB
:10016000D66EF294D58E818ECD90FE0ECF6E6F0E30
:10017000CE6E9E90CD8009D0818ECD90FE0ECF6E3A
:100180006F0ECE6E9E90CD8000D0A32B03D09E909C
:10019000CD90819EE552E5CFDAFF1100D9CFE6FF81
:1001A000E1CFD9FFFE0EDB50A96EA69EA69CA680CD
:1001B000A85000D0E552E7CFD9FF1200D9CFE6FF13
:1001C000E1CFD9FFFE0EDB50A96EFD0EDB50A86E0D
:1001D000A69EA69CA684F29E550EA76EAA0EA76E9A
:1001E000A682F28EA1A8FED7A198A694E552E7CFE9
:1001F000D9FF1200D9CFE6FFE1CFD9FFE652FE0EBC
:10020000DB50DF6ED9CFE9FFDACFEAFFEF50800B8A
:1002100002E0828A01D0829A0000808A809AD9CF37
:10022000E9FFDACFEAFFEF50400B02E0828A01D00B
:10023000829A0000808A809AD9CFE9FFDACFEAFF5C
:10024000EF50200B02E0828A01D0829A0000808A5F
:10025000809AD9CFE9FFDACFEAFFEF50100B02E026
:10026000828A01D0829A0000808A809AD9CFE9FFE1
:10027000DACFEAFFEF50080B02E0828A01D0829ABF
:100280000000808A809AD9CFE9FFDACFEAFFEF50E9
:10029000040B02E0828A01D0829A0000808A809A50
:1002A000D9CFE9FFDACFEAFFEF50020B02E0828AF2
:1002B00001D0829A0000808A809AD9CFE9FFDACFF4
:1002C000EAFFEF50010B02E0828A01D0829A00001F
:1002D000808A809AE552E552E7CFD9FF1200D9CF44
:1002E000E6FFE1CFD9FFE652948AD9CFE9FFDACF12
:1002F000EAFF8250200B02E0EF8E01D0EF9E808A51
:10030000809AD9CFE9FFDACFEAFF8250200B02E0D2
:10031000EF8C01D0EF9C808A809AD9CFE9FFDACFA9
:10032000EAFF8250200B02E0EF8A01D0EF9A808A28
:10033000809AD9CFE9FFDACFEAFF8250200B02E0A2
:10034000EF8801D0EF98808A809AD9CFE9FFDACF81
:10035000EAFF8250200B02E0EF8601D0EF96808A00
:10036000809AD9CFE9FFDACFEAFF8250200B02E072
:10037000EF8401D0EF94808A809AD9CFE9FFDACF59
:10038000EAFF8250200B02E0EF8201D0EF92808AD8
:10039000809AD9CFE9FFDACFEAFF8250200B02E042
:1003A000EF8001D0EF90808A809A949ADF5000D03D
:1003B000E552E552E7CFD9FF12008098450EE66E70
:1003C00019DFE5528CDF0001796F89DF0001616F71
:1003D00086DF0001626F83DF0001636F80DF000151
:1003E000646F7DDF0001696F7ADF00016A6F77DF7C
:1003F00000016B6F74DF00016C6F71DF00016D6FC6
:100400006EDF00016E6F6BDF00016F6F68DF000150
:10041000706F65DF0001716F62DF0001726F5FDF77
:100420000001736F5CDF0001746F59DF0001756FAD
:1004300056DF0001766F53DF0001776F50DF000158
:10044000786F8088CA0ED8806955080E6A5504E214
:10045000CA0E696F080E6A6FEE0E695D020E6A5968
:1004600004E2EE0E696F020E6A6FCA0ED8806B55F9
:10047000080E6C5504E2CA0E6B6F080E6C6FEE0E20
:100480006B5D020E6C5904E2EE0E6B6F020E6C6F28
:10049000CA0ED8806D55080E6E5504E2CA0E6D6FF7
:1004A000080E6E6FEE0E6D5D020E6E5904E2EE0EDA
:1004B0006D6F020E6E6FCA0ED8806F55080E7055A4
:1004C00004E2CA0E6F6F080E706FEE0E6F5D020EC3
:1004D000705904E2EE0E6F6F020E706FCA0ED88074
:1004E0007155080E725504E2CA0E716F080E726FD4
:1004F000EE0E715D020E725904E2EE0E716F020E85
:10050000726FCA0ED8807355080E745504E2CA0E75
:10051000736F080E746FEE0E735D020E745904E271
:10052000EE0E736F020E746FCA0ED8807555080EEA
:10053000765504E2CA0E756F080E766FEE0E755D85
:10054000020E765904E2EE0E756F020E766FCA0E39
:10055000D8807755080E785504E2CA0E776F080EDA
:10056000786FEE0E775D020E785904E2EE0E776F2B
:10057000020E786F1200D9CFE6FFE1CFD9FF020E4D
:10058000E1268098E66A36DEE552E66A33DEE55219
:1005900080888098060EE66E2DDEE552540EE66EDB
:1005A00029DEE552750EE66E25DEE552C50EE66ED5
:1005B00021DEE5522A0EE66E1DDEE552808800013E
:1005C000616B626B636B646B8098460EE66E12DE45
:1005D000E55285DE0001616F82DE0001626F7FDE21
:1005E0000001636F7CDE0001646F8088DF6A320E79
:1005F000DF5C1AE2DF50F76A600FF66E0E0EF7222C
:100600000800010EF5CFDBFFDB50FF080BE0809800
:10061000DFCFE6FFEFDDE552010EDBCFE6FFEADDDF
:10062000E5528088DF2AE3D78098020EE66EE2DD8D
:10063000E552010EE66EDEDDE5528088010EDB68D4
:10064000DBA00CD08098420EE66ED4DDE55247DE8A
:10065000E76E010EE7CFDBFF8088F2D78098240E8B
:10066000E66EC8DDE552130EE66EC4DDE552808805
:100670008098260EE66EBEDDE5523B0EE66EBADDD4
:10068000E552808880980F0EE66EB4DDE552E66A8A
:10069000B1DDE55280888098020EE66EABDDE55252
:1006A000020EE66EA7DDE5528088010EDB68DBA056
:1006B0000CD08098420EE66E9DDDE55210DEE76EAE
:1006C000010EE7CFDBFF8088F2D780980F0EE66E31
:1006D00091DDE552A00EE66E8DDDE55280888098B2
:1006E000020EE66E87DDE552020EE66E83DDE55210
:1006F0008088010EDB68DBA00CD08098420EE66E8D
:1007000079DDE552ECDDE76E010EE7CFDBFF808897
:10071000F2D78098250EE66E6DDDE552080EE66E86
:1007200069DDE55280888098A00EE66E63DDE552B3
:100730008088020EE15C02E2E16AE552E16EE55278
:10074000E7CFD9FF1200D9CFE6FFE1CFD9FF030EE3
:10075000E126DF6AD00EF36E010EF3CFDBFF070E4A
:10076000F36E020EF3CFDBFFB190F90EB36EF10E14
:10077000B26EA192B180DF5001E08BD0010EDBCFD1
:1007800000F0020EDBCF01F0013404E2005000085B
:10079000000E015401E37DD0010EDB06020E01E2E2
:1007A000DB06300EE76E010EDBCF00F0020EDBCF72
:1007B00001F0E7500016016A300E001801E1015007
:1007C00002E1828C01D0829C8098A00EE66E12DD40
:1007D000E55280888098F00EE66E0CDDE552808848
:1007E00080980F0EE66E06DDE552E66A03DDE552FF
:1007F00080888098C00EE66EFDDCE5528088A150AE
:10080000020B04E18250010B01E0F9D7B190F90E1F
:10081000B36EF10EB26EA192B18082B039D08098E1
:10082000400EE66EE7DCE5525ADD0001606F80881D
:100830006051200B2DE16051400B2AE1BEDDAA0E74
:100840000001795D25E1010EDF6E61C0E6FFE66A19
:10085000B5DCE552E55262C0E6FF010EE66EAEDCA5
:10086000E552E55263C0E6FF020EE66EA7DCE552F4
:10087000E55264C0E6FF030EE66EA0DCE552E552E9
:1008800061C065F062C066F063C067F064C068F084
:1008900072D7010EDBCF00F0020EDBCF01F0013486
:1008A00004E200500008000E015422E2010EDB06B3
:1008B000020E01E2DB06C00EE76E010EDBCF00F098
:1008C000020EDBCF01F0E7500016016AC00E0018DF
:1008D00001E1015002E1828C01D0829CB190F90EBD
:1008E000B36EF10EB26EA192B180A1A2FED7D1D7A4
:1008F000DF5017E1E66A52DCE5520001656F010E38
:10090000E66E4CDCE5520001666F020EE66E46DCD8
:10091000E5520001676F030EE66E40DCE552000110
:10092000686F030EE15C02E2E16AE552E16EE552B6
:10093000E7CFD9FF120000019D2B100E9D5D01E154
:100940009D6B9E51100DF3CF04F0F4CF05F0920E85
:1009500004260E0E05229D510F010424F66E000E92
:100960000520F76E0800F550026E036A00019F51E2
:10097000025C006EA0510358016E00C09CF0120092
:10098000D388D38AD38C806A816A826A828C949C51
:1009900080889298828A949A809A929A939C939A49
:1009A00093989494949294989496939E7E6A7F6A76
:1009B0009280F19E7780040EE66ECEEC00F0E55258
:1009C00000017A6F050EE66ECEEC00F0E5520001F4
:1009D0007B6F060EE66ECEEC00F0E55200017C6FF8
:1009E000070EE66ECEEC00F0E55200017D6F080EBA
:1009F000E66ECEEC00F0E55200017E6F090EE66E69
:100A0000CEEC00F0E55200017F6F0A0EE66ECEECF0
:100A100000F0E5520001806F0B0EE66ECEEC00F0A8
:100A2000E5520001816F0C0EE66ECEEC00F0E5524F
:100A30000001826F0D0EE66ECEEC00F0E552000173
:100A4000836F0E0EE66ECEEC00F0E5520001846F6F
:100A50000F0EE66ECEEC00F0E5520001856F100E31
:100A6000E66ECEEC00F0E5520001866F110EE66EE8
:100A7000CEEC00F0E5520001876F120EE66ECEEC70
:100A800000F0E5520001886F130EE66ECEEC00F028
:100A9000E5520001896F840E8A6F020E8B6FD56A52
:100AA000D580F294F28ACD6ACD8ECD8A9E909D80BB
:100AB0009F80F90ECB6ECA6ACA8CCA86CA829E9281
:100AC0009D829F82F28CF28EB16AB18EB18AA19220
:100AD000DC0E8C6F050E8D6FDC0E8E6F050E8F6F2A
:100AE000E80E906F030E916FDC0E926F050E936F00
:100AF000DC0E946F050E956FDC0E966F050E976FEA
:100B0000DC0E986F050E996FDC0E9A6F050E9B6FC9
:100B1000CA84B1903C0EB36EAF0EB26EA192B1809A
:100B2000A1A2FED728DD0FDE00019D6B0F0E65151B
:100B30009E6FF00E6515E8380F0B9F6FA06B090EC6
:100B4000D8809F55000EA05503E2090E9F6FA06B41
:100B50009F2B000EA023B190F90EB36EF10EB26E72
:100B6000A192B180E8DE8098A00EE66EFAEC00F06B
:100B7000E55280888098F00EE66EFAEC00F0E552BF
:100B8000808880980F0EE66EFAEC00F0E5529CC06B
:100B9000E6FFFAEC00F0E55280888098C00EE66E21
:100BA000FAEC00F0E5528088A150020B04E182507B
:100BB000010B01E0F9D7B190F90EB36EF10EB26EF0
:100BC000A192B18082B064D08098400EE66EFAECBB
:100BD00000F0E5526FEC01F00001606F8088605119
:100BE000200B54E16051400B51E1DDEC01F0550E5A
:100BF0000001795D49E1650EE96E000EEA6EEE5086
:100C0000611909E1EE50621906E1EE50631903E142
:100C1000EE50641900E136E1F29E69C08CF06AC0C2
:100C20008DF0F28EF29E6BC08EF06CC08FF0F28E63
:100C3000F29E6DC090F06EC091F0F28EF29E6FC089
:100C400092F070C093F0F28EF29E71C094F072C078
:100C500095F0F28EF29E73C096F074C097F0F28E0B
:100C6000F29E75C098F076C099F0F28EF29E77C031
:100C70009AF078C09BF0F28E828C840E8A6F020EFE
:100C80008B6F01D0829C01D0829C01D0829C01D0CC
:100C9000829C00018A07000E8B5B800E8B1530E072
:100CA000F29E7AC08CF07BC08DF0F28EF29E7CC0FA
:100CB0008EF07DC08FF0F28EF29E7EC090F07FC0ED
:100CC00091F0F28EF29E80C092F081C093F0F28E8D
:100CD000F29E82C094F083C095F0F28EF29E84C0A2
:100CE00096F085C097F0F28EF29E86C098F087C08D
:100CF00099F0F28EF29E88C09AF089C09BF0F28E35
:100D000080B0ACD0829C69C07AF06AC07BF06BC0C6
:100D10007CF06CC07DF06DC07EF06EC07FF06FC067
:100D200080F070C081F071C082F072C083F073C037
:100D300084F074C085F075C086F076C087F077C007
:100D400088F078C089F07AC0E6FF040EE66EDEEC2B
:100D500000F0E552E5527BC0E6FF050EE66EDEECE4
:100D600000F0E552E5527CC0E6FF060EE66EDEECD2
:100D700000F0E552E5527DC0E6FF070EE66EDEECC0
:100D800000F0E552E5527EC0E6FF080EE66EDEECAE
:100D900000F0E552E5527FC0E6FF090EE66EDEEC9C
:100DA00000F0E552E55280C0E6FF0A0EE66EDEEC8A
:100DB00000F0E552E55281C0E6FF0B0EE66EDEEC78
:100DC00000F0E552E55282C0E6FF0C0EE66EDEEC66
:100DD00000F0E552E55283C0E6FF0D0EE66EDEEC54
:100DE00000F0E552E55284C0E6FF0E0EE66EDEEC42
:100DF00000F0E552E55285C0E6FF0F0EE66EDEEC30
:100E000000F0E552E55286C0E6FF100EE66EDEEC1D
:100E100000F0E552E55287C0E6FF110EE66EDEEC0B
:100E200000F0E552E55288C0E6FF120EE66EDEECF9
:100E300000F0E552E55289C0E6FF130EE66EDEECE7
:100E400000F0E552E55280A0FED7B1903C0EB36EA3
:100E5000AF0EB26EA192B180A1A2FED783D61200CE
:100E6000FF42001400FFFF000000000121050050B8
:100E70009E4B0002162B1200628080000A32C30FC4
:100E800013C300FF00003B00174780030145180013
:100E9000010F0A5A14641E6E287832823C8C4696E2
:100EA00050A0A05096468C3C823278286E1E641466
:100EB0005A0A0A5A50A0146446961E6E3C8C287832
:100EC0003282823278288C3C6E1E96466414A05082
:100ED0005A0A28780A5A50A014641E6E3C8C32823A
:100EE0004696964682328C3C6E1E6414A0505A0A76
:100EF000782850A028780A5A1E6E3C8C328246967A
:100F000014646414964682328C3C6E1E5A0A782809
:100F1000A05050A046963C8C28780A5A32821E6E09
:100F2000146464146E1E82325A0A78288C3C9646E9
:100F3000A05046963C8C50A028780A5A1E6E3282E9
:100F40001464641482326E1E5A0A7828A0508C3CB5
:100F5000964646960A5A3C8C146450A028781E6E19
:100F6000328282326E1E7828A05064148C3C5A0A59
:100F7000964646960A5A50A03C8C28781E6E3282BD
:100F80001464641482326E1E78288C3CA0505A0A75
:100F90009646060EF66E000EF76E000EF86E000115
:100FA0000900F550A96F0900F550AA6F03E1A96780
:100FB00001D03DD00900F550A46F0900F550A56F90
:100FC0000900F550A66F09000900F550E96E090007
:100FD000F550EA6E090009000900F550A76F0900F5
:100FE000F550A86F09000900F6CFABF0F7CFACF0D1
:100FF000F8CFADF0A4C0F6FFA5C0F7FFA6C0F8FF7C
:101000000001A75302E1A85307E00900F550EE6E76
:10101000A707F8E2A807F9D7ABC0F6FFACC0F7FF07
:10102000ADC0F8FF0001A907000EAA5BBFD71200F0
:10103000000EF36E00EE00F0020E01D81200EA601E
:1010400002D0EE6AFCD7F350E9601200EE6AFCD7DA
:1010500011EE00F021EE00F0F86A079CC9EC07F0F1
:1010600036EC08F0C0EC04F0FBD712001200FFFFD2
:10107000FFFFFFFFFFFFFFFFFFFFFFFFFFFFFFFF80
:10108000FFFFFFFFFFFFFFFFFFFFFFFFFFFFFFFF70
:10109000FFFFFFFFFFFFFFFFFFFFFFFFFFFFFFFF60
:1010A000FFFFFFFFFFFFFFFFFFFFFFFFFFFFFFFF50
:0200000400F00A
:10000000B2A10000DC05DC05E803DC05DC05DC054D
:10001000DC05DC05FFFFFFFFFFFFFFFFFFFFFFFF2A
:10002000FFFFFFFFFFFFFFFFFFFFFFFFFFFFFFFFE0
:10003000FFFFFFFFFFFFFFFFFFFFFFFFFFFFFFFFD0
:10004000FFFFFFFFFFFFFFFFFFFFFFFFFFFFFFFFC0
:10005000FFFFFFFFFFFFFFFFFFFFFFFFFFFFFFFFB0
:10006000FFFFFFFFFFFFFFFFFFFFFFFFFFFFFFFFA0
:10007000FFFFFFFFFFFFFFFFFFFFFFFFFFFFFFFF90
:10008000FFFFFFFFFFFFFFFFFFFFFFFFFFFFFFFF80
:10009000FFFFFFFFFFFFFFFFFFFFFFFFFFFFFFFF70
:1000A000FFFFFFFFFFFFFFFFFFFFFFFFFFFFFFFF60
:1000B000FFFFFFFFFFFFFFFFFFFFFFFFFFFFFFFF50
:1000C000FFFFFFFFFFFFFFFFFFFFFFFFFFFFFFFF40
:1000D000FFFFFFFFFFFFFFFFFFFFFFFFFFFFFFFF30
:1000E000FFFFFFFFFFFFFFFFFFFFFFFFFFFFFFFF20
:1000F000FFFFFFFFFFFFFFFFFFFFFFFFFFFFFFFF10
:020000040030CA
:0E0000000008191E0000800003C003E003404A
:020000040020DA
:08000000FFFFFFFFFFFFFFFF00
:00000001FF
